:020000040000FA
:0A0000000000000097EF01F0AAD104
:08001800F7D1076A066EFF0E26
:100020000626072200D0D8A01200030E056EE60EA9
:1000300002D8F5D7056AFE0F046EE86A055AD8A003
:1000400012000000040600D0F8D7800E1C1A1B50C6
:10005000175C206E11E2206C17501BC017F01B6E4E
:1000600018501CC018F01C6E19501DC019F01D6EE0
:100070001A501EC01AF01E6E1A0E206074D01B5249
:1000800072E01F6A1850226E1C18236E188E1C8E88
:10009000080E205E08E31EC01FF01DC01EF01CC02D
:1000A0001DF01C6AF5D7202607E0D8901C321D32BF
:1000B0001E321F32202EF9D723AE33D01E501A5EC7
:1000C0001D50195A1C50185A07E2D880000E1A56B3
:1000D00019561856800E221A1F6C04E01A06000EDC
:1000E000195A185A040E206E18660DD019C018F04F
:1000F0001AC019F01FC01AF01F6A080E175E29E314
:10010000202EF2D726D018BE08D0D8901F361A3627
:1001100019361836172EF7D71CD01FAE22D01F6AFB
:100120000FD01E501A261D5019221C50182206E30B
:10013000183219321A321F32174A0DD01FAE11D0A1
:100140001A3E0FD0193E0DD0183E0BD0D8801A9011
:10015000EFD7176A02D0218217681A6A196A800ECF
:10016000186E22AE189E1A5012001850166E1C18E7
:10017000236E1750D8A41B503AE017267E0E03E3D7
:10018000175E03E336D0175E31E31AC014F019C0CE
:1001900015F0168E1C8E1A6A196A186A180E226ECD
:1001A00016321532143206E31E501A261D5019223B
:1001B0001C501822183219321A32222EF1D718BECA
:1001C00007D01A3619361836175210E017061634AB
:1001D00016E31A3E14D0193E12D0183E10D0D88023
:1001E000183219321A32173E0AD003D02184176A06
:1001F00002D0218217681A6A196A800E186E23AE1F
:10020000189E1A50120017C022F018501AC018F089
:100210001A6E1A3622321A32216A1A36223602E34E
:100220002184217E06E12180226A1A6A196A186AED
:100230000BD0222803E0D8801A3206D0D8901A3288
:1002400002E1218201D0218621B604D021A20FD063
:1002500021B407D07F0E1A6EFF0E196E186E176E3E
:1002600023D0800E1A6E01D01A6A000EF6D721B084
:10027000FBD7176A9F0E2260EBD77E0E2264F4D75D
:100280009E0E225C07E0D8901A32193218321732CB
:10029000222AF6D721A408D0D880000E1756185667
:1002A00019561A561AAEE0D717501200176E186A70
:1002B000196A1A6A239E0AD0239E1AAE07D0D880E4
:1002C000000E1756185619561A56238E960E226E81
:1002D0001A5209E0080E222618C017F019C018F0AB
:1002E0001AC019F011D019520FE1080E225E1850F1
:1002F00007E1080E225E175002E11A5010D0176A6B
:10030000196E17C018F0176A19BE06D0D8901736A4
:10031000183619362206F8D723AE199E225017C078
:100320001AF0176E195018C019F0186E1200400E0E
:10033000216E4F0EAF6E240EAC6E900EAB6E0001B0
:100340000F0EC16E070EB46EC69AC00E926EE00E0E
:10035000936EC00E946E956AE80E966E6CD0F2A401
:1003600003D0F294817A11009EAA19D0060EAB1424
:1003700012E1E2CF7DF0E1CF7CF07E2A11EE00F0B9
:100380007E50E126000EE222AECFE7FF7DC0E2FF05
:100390007CC0E1FF1100AE50AE50AB98AB881100AD
:1003A0007E507F5C14E07F2AEACF05F0E9CF04F0AD
:1003B00001EE00F07F50E926000EEA22EF50046EB5
:1003C00005C0EAFF04C0E9FFD880120004D0E86845
:1003D000046ED8A0120012007E6A7F6A9D8A9F8AEE
:1003E000F28EF28C12009D9A01EE00F0010EF46E76
:1003F000F36AF306000EF45AEE6AF450F310F9E1D2
:100400007E6A7F6A9D8A1200F29EE0CFC9F4D8CF3F
:10041000CAF4E8CFCBF4F28E0001A192F29EC9C4D7
:10042000E0FFCAC4D8FFCBC4E8FFF28E10009EA83C
:10043000FED7AD6E1200939A8A8A0A0E0DEC00F078
:10044000939A8A9A95928C92929289929294899494
:10045000929689969290899092988998929A899A80
:1004600096908D9096928D9296948D9493988A986A
:1004700093968A9693948A9493928A9293908A9070
:10048000959E8C9E959C8C9C959A8C9A95988C9810
:10049000949A8B9A94988B9895968C9695948C9424
:1004A00094908B9094928B9294948B9495908C9042
:1004B00094968B9695928C925C6A5B6A5A6A596A9A
:1004C000576A566A00EEA0F0280EEE68E82EFDD7B7
:1004D000586A966B976B986B996B9A6B9B6B9C6B3E
:1004E0009D6B9E6B9F6B836B826B856B846B876B45
:1004F000866B896B886B8B6B8A6B8D6B8C6B8F6B50
:100500008E6B916B906B936B926B956B946B5E6A39
:100510005D6A606A5F6A626A616A646A636A666A7F
:10052000656A686A676A6A6A696A6C6A6B6A6E6A2F
:100530006D6A706A6F6AC86B4FDF55DFCD6AF294DF
:10054000F28A870ED56EB16AA192A082D08EA29255
:10055000B10EB16E20EC0CF022EC0EF0752AE86AB8
:1005600075B2010F76B0010806E17670712A000EAF
:1005700072227322742214DF246EC50E245C06E3FB
:10058000FE0E245C01E2256AF3EF06F024AE29D0CA
:10059000256A840E245C05E124C025F02668816963
:1005A0001ED0940E245C05E124C025F0276828683D
:1005B00016D0A40E245C05E124C025F029682A6821
:1005C0000ED0B40E245C05E124C025F02B682C6805
:1005D00006D0C40E245C03E124C025F02D68F1EFA1
:1005E00006F0255204E1F3EF06F0F1EF06F0840E79
:1005F000255CD8A48BD0262803E124C026F082D025
:1006000024C081F03C0E265C08E1569059905BB006
:1006100002D0899401D0899272D03D0E265C08E107
:10062000569259925BB002D0899001D0899667D0DA
:100630003E0E265C08E1569459945BB402D089982A
:1006400001D08D925CD03F0E265C08E156965996FB
:100650005BB602D08D9001D08D9251D0400E265CB9
:1006600008E1569859985BB802D08D9401D08A98C9
:1006700046D0410E265C08E1569A599A5BBA02D0E0
:100680008A9601D08A943BD0420E265C08E1569CA3
:10069000599C5BBC02D08A9201D08A9030D0430E24
:1006A000265C08E1569E599E5BBE02D08C9E01D00E
:1006B0008C9C25D0440E265C08E157905A905CB083
:1006C00002D08C9A01D08C981AD0450E265C08E195
:1006D00057925A925CB202D08B9A01D08B980FD06D
:1006E000780E265C05E18C902668F3EF06F007D0C3
:1006F000790E265C04E18B962668F3EF06F02668F7
:10070000F1EF06F0F3EF06F0F1EF06F0940E255C42
:10071000D8A4CBEF06F0272804E124C027F0C9EFC6
:1007200006F024C028F02852D8A481D03C0E275CC3
:1007300008E1569059905BB002D0899401D089921B
:1007400072D03D0E275C08E1569259925BB002D000
:10075000899001D0899667D03E0E275C08E15694B7
:1007600059945BB402D0899801D08D925CD03F0E31
:10077000275C08E1569659965BB602D08D9001D061
:100780008D9251D0400E275C08E1569859985BB87D
:1007900002D08D9401D08A9846D0410E275C08E1A2
:1007A000569A599A5BBA02D08A9601D08A943BD065
:1007B000420E275C08E1569C599C5BBC02D08A9291
:1007C00001D08A9030D0430E275C08E1569E599E96
:1007D0005BBE02D08C9E01D08C9C25D0440E275C41
:1007E00008E157905A905CB002D08C9A01D08C9856
:1007F0001AD0450E275C08E157925A925CB202D09B
:100800008B9A01D08B980FD0780E275C05E18C90E5
:100810002668F3EF06F007D0790E275C04E18B968B
:100820002668F3EF06F0F1EF06F0C9EF06F03C0E94
:10083000275CD8A440D05BB003D08994898202D0D1
:10084000899289845B70568002EEC9F0D890283472
:10085000E926000EEA22EECF5DF0EFCF5EF05D50AC
:100860007124006E5E507220016E000E7320026EC5
:10087000000E7420036E03C0A3F002C0A2F001C0FA
:10088000A1F000C0A0F0965313E0598003EEC9F028
:10089000D8909635E926000EEA22EECF00F0EFCF91
:1008A00001F05D50005C826F5E500158836F01D093
:1008B0005990C7EF06F03D0E275CD8A440D05BB23C
:1008C00003D08990898602D0899689805B7256828E
:1008D00002EEC9F0D8902834E926000EEA22EECFC5
:1008E0005FF0EFCF60F05F507124006E60507220B7
:1008F000016E000E7320026E000E7420036E03C0A2
:10090000A7F002C0A6F001C0A5F000C0A4F0975364
:1009100013E0598203EEC9F0D8909735E926000E0E
:10092000EA22EECF00F0EFCF01F05F50005C846F61
:1009300060500158856F01D05992C7EF06F03E0E06
:10094000275CD8A43FD05BB403D08998898A02D0B1
:10095000899A89885B74568402EEC9F0D89028344D
:10096000E926000EEA22EECF61F0EFCF62F061508F
:100970007124006E62507220016E000E7320026EB0
:10098000000E7420036E03C0ABF002C0AAF001C0D9
:10099000A9F000C0A8F0985313E0598403EEC9F001
:1009A000D8909835E926000EEA22EECF00F0EFCF7E
:1009B00001F06150005C866F62500158876F01D072
:1009C0005994E5D13F0E275CD8A43FD05BB603D045
:1009D0008D908D8202D08D928D805B76568602EE50
:1009E000C9F0D8902834E926000EEA22EECF63F051
:1009F000EFCF64F063507124006E64507220016E7A
:100A0000000E7320026E000E7420036E03C0AFF060
:100A100002C0AEF001C0ADF000C0ACF0995313E0DD
:100A2000598603EEC9F0D8909935E926000EEA22DE
:100A3000EECF00F0EFCF01F06350005C886F6450A0
:100A40000158896F01D05996A2D1400E275CD8A4D5
:100A50003FD05BB803D08D948A8802D08A988D8469
:100A60005B78568802EEC9F0D8902834E926000E4B
:100A7000EA22EECF65F0EFCF66F065507124006E8C
:100A800066507220016E000E7320026E000E7420FC
:100A9000036E03C0B3F002C0B2F001C0B1F000C0F9
:100AA000B0F09A5313E0598803EEC9F0D8909A3504
:100AB000E926000EEA22EECF00F0EFCF01F06550FC
:100AC000005C8A6F665001588B6F01D059985FD1D6
:100AD000410E275CD8A43FD05BBA03D08A968A84A3
:100AE00002D08A948A865B7A568A02EEC9F0D89040
:100AF0002834E926000EEA22EECF67F0EFCF68F047
:100B000067507124006E68507220016E000E7320D1
:100B1000026E000E7420036E03C0B7F002C0B6F080
:100B200001C0B5F000C0B4F09B5313E0598A03EE46
:100B3000C9F0D8909B35E926000EEA22EECF00F0EE
:100B4000EFCF01F06750005C8C6F685001588D6FDB
:100B500001D0599A1CD1420E275CD8A43FD05BBC6F
:100B600003D08A928A8002D08A908A825B7C568CDB
:100B700002EEC9F0D8902834E926000EEA22EECF22
:100B800069F0EFCF6AF069507124006E6A507220EC
:100B9000016E000E7320026E000E7420036E03C0FF
:100BA000BBF002C0BAF001C0B9F000C0B8F09C536D
:100BB00013E0598C03EEC9F0D8909C35E926000E5D
:100BC000EA22EECF00F0EFCF01F06950005C8E6FAB
:100BD0006A5001588F6F01D0599CD9D0430E275CC1
:100BE000D8A43FD05BBE03D08C9E8C8C02D08C9C52
:100BF0008C8E5B7E568E02EEC9F0D8902834E926A2
:100C0000000EEA22EECF6BF0EFCF6CF06B50712448
:100C1000006E6C507220016E000E7320026E000E8A
:100C20007420036E03C0BFF002C0BEF001C0BDF06F
:100C300000C0BCF09D5313E0598E03EEC9F0D8906C
:100C40009D35E926000EEA22EECF00F0EFCF01F04D
:100C50006B50005C906F6C500158916F01D0599EA1
:100C600096D0440E275CD8A43FD05CB003D08C9AB9
:100C70008C8802D08C988C8A5C70578002EEC9F008
:100C8000D8902834E926000EEA22EECF6DF0EFCF9F
:100C90006EF06D507124006E6E507220016E000E69
:100CA0007320026E000E7420036E03C0C3F002C0F6
:100CB000C2F001C0C1F000C0C0F09E5313E05A80E2
:100CC00003EEC9F0D8909E35E926000EEA22EECF59
:100CD00000F0EFCF01F06D50005C926F6E50015844
:100CE000936F01D05A9053D0450E275CD8A43FD0C3
:100CF0005CB203D08B9A8B8802D08B988B8A5C7203
:100D0000578202EEC9F0D8902834E926000EEA2274
:100D1000EECF6FF0EFCF70F06F507124006E705017
:100D20007220016E000E7320026E000E7420036E9E
:100D300003C0C7F002C0C6F001C0C5F000C0C4F0D7
:100D40009F5313E05A8203EEC9F0D8909F35E926ED
:100D5000000EEA22EECF00F0EFCF01F06F50005C02
:100D6000946F70500158956F01D05A9210D0780E40
:100D7000275C04E18C80276836D009D0790E275C87
:100D800004E18B8627682FD002D027682CD02768F3
:100D900028D029D026D0A40E255C0BE1292803E118
:100DA00024C029F004D024C02AF00AEC0AF01BD099
:100DB00018D0B40E255C0BE12B2803E124C02BF0E6
:100DC00004D024C02CF006EC0BF00DD00AD0C40ED9
:100DD000255C07E12D2804E124C02DF0F1EC0AF098
:100DE00002D0D0EC09F00A0E7B5CD8B0C8EF09F055
:100DF0007750715C78507258795073587A507458A3
:100E0000D8A0B7EF09F07A8E7B52D8A442D05BB05D
:100E100002D0899401D0899259B006D05690A36926
:100E2000A269A169A06933D056A016D0825171245D
:100E3000006E83517220016E000E7320026E000E50
:100E40007420036E03C0A3F002C0A2F001C0A1F0A1
:100E500000C0A0F056901BD05BB002D0898201D0B8
:100E600089845B705D507124006E5E507220016E4B
:100E7000000E7320026E000E7420036E03C0A3F0F8
:100E800002C0A2F001C0A1F000C0A0F05680B6EFF1
:100E900009F0010E7B5CD8A442D05BB202D08990ED
:100EA00001D0899659B206D05692A769A669A5695C
:100EB000A46933D056A216D084517124006E855196
:100EC0007220016E000E7320026E000E7420036EFD
:100ED00003C0A7F002C0A6F001C0A5F000C0A4F0B6
:100EE00056921BD05BB202D0898601D089805B729A
:100EF0005F507124006E60507220016E000E7320EE
:100F0000026E000E7420036E03C0A7F002C0A6F0AC
:100F100001C0A5F000C0A4F05682B6EF09F0020EA1
:100F20007B5CD8A441D05BB402D0899801D0899A67
:100F300059B406D05694AB69AA69A969A86933D097
:100F400056A416D086517124006E87517220016E0E
:100F5000000E7320026E000E7420036E03C0ABF00F
:100F600002C0AAF001C0A9F000C0A8F056941BD09E
:100F70005BB402D0898A01D089885B746150712486
:100F8000006E62507220016E000E7320026E000E21
:100F90007420036E03C0ABF002C0AAF001C0A9F038
:100FA00000C0A8F05684E2D1030E7B5CD8A441D0E7
:100FB0005BB602D08D9001D08D9259B606D0569670
:100FC000AF69AE69AD69AC6933D056A616D0885109
:100FD0007124006E89517220016E000E7320026E22
:100FE000000E7420036E03C0AFF002C0AEF001C06B
:100FF000ADF000C0ACF056961BD05BB602D08D822F
:1010000001D08D805B7663507124006E6450722035
:10101000016E000E7320026E000E7420036E03C07A
:10102000AFF002C0AEF001C0ADF000C0ACF056862B
:101030009DD1040E7B5CD8A441D05BB802D08D94C6
:1010400001D08A9859B806D05698B369B269B16987
:10105000B06933D056A816D08A517124006E8B51D6
:101060007220016E000E7320026E000E7420036E5B
:1010700003C0B3F002C0B2F001C0B1F000C0B0F0E4
:1010800056981BD05BB802D08A8801D08D845B78DB
:1010900065507124006E66507220016E000E732040
:1010A000026E000E7420036E03C0B3F002C0B2F0F3
:1010B00001C0B1F000C0B0F0568858D1050E7B5C7D
:1010C000D8A441D05BBA02D08A9601D08A9459BA8A
:1010D00006D0569AB769B669B569B46933D056AACD
:1010E00016D08C517124006E8D517220016E000E4D
:1010F0007320026E000E7420036E03C0B7F002C0AE
:10110000B6F001C0B5F000C0B4F0569A1BD05BBA7F
:1011100002D08A8401D08A865B7A67507124006E7F
:1011200068507220016E000E7320026E000E742053
:10113000036E03C0B7F002C0B6F001C0B5F000C046
:10114000B4F0568A13D1060E7B5CD8A441D05BBCA8
:1011500002D08A9201D08A9059BC06D0569CBB69B5
:10116000BA69B969B86933D056AC16D08E517124BA
:10117000006E8F517220016E000E7320026E000E01
:101180007420036E03C0BBF002C0BAF001C0B9F016
:1011900000C0B8F0569C1BD05BBC02D08A8001D046
:1011A0008A825B7C69507124006E6A507220016EE5
:1011B000000E7320026E000E7420036E03C0BBF09D
:1011C00002C0BAF001C0B9F000C0B8F0568CCED061
:1011D000070E7B5CD8A441D05BBE02D08C9E01D0B0
:1011E0008C9C59BE06D0569EBF69BE69BD69BC695C
:1011F00033D056AE16D090517124006E91517220AA
:10120000016E000E7320026E000E7420036E03C088
:10121000BFF002C0BEF001C0BDF000C0BCF0569EE1
:101220001BD05BBE02D08C8C01D08C8E5B7E6B5051
:101230007124006E6C507220016E000E7320026EDD
:10124000000E7420036E03C0BFF002C0BEF001C0E8
:10125000BDF000C0BCF0568E89D0080E7B5CD8A4CF
:1012600041D05CB002D08C9A01D08C985AB006D094
:101270005790C369C269C169C06933D057A016D0FD
:1012800092517124006E93517220016E000E7320F2
:10129000026E000E7420036E03C0C3F002C0C2F0E1
:1012A00001C0C1F000C0C0F057901BD05CB002D0AC
:1012B0008C8801D08C8A5C706D507124006E6E50E9
:1012C0007220016E000E7320026E000E7420036EF9
:1012D00003C0C3F002C0C2F001C0C1F000C0C0F042
:1012E000578044D0090E7B5CD8A440D05CB202D0B9
:1012F0008B9A01D08B985AB206D05792C769C669AB
:10130000C569C46933D057A216D094517124006EB8
:1013100095517220016E000E7320026E000E742033
:10132000036E03C0C7F002C0C6F001C0C5F000C024
:10133000C4F057921BD05CB202D08B8801D08B8A4C
:101340005C726F507124006E70507220016E000E3E
:101350007320026E000E7420036E03C0C7F002C03B
:10136000C6F001C0C5F000C0C4F0578219D874AEF1
:101370000ED0746A736A726A716A576A566A5A6AD8
:10138000596A00EEA0F0280EEE68E82EFDD706D0D0
:1013900074AE04D0746A736A726A716AAEEF02F056
:1013A0007B687A8E806B0A0E805D33E2D890803540
:1013B000E96EEA6AEA36E936EA36A00EE926000E58
:1013C000EA22EFCF00F0ECCF01F0ECCF02F0ECCF4F
:1013D00003F07750005C78500158795002587A50E9
:1013E000035815E2D8908035E96EEA6AEA36E936A4
:1013F000EA36A00EE926000EEA22EFCF77F0ECCF16
:1014000078F0ECCF79F0ECCF7AF080C07BF0802BD5
:10141000CAE312003C0E295C14E12AC096F09653F0
:101420000CE003EEC9F0D8909635E926000EEA22CA
:10143000EECF82F0EFCF83F003D0836B826B5990B5
:10144000CED03D0E295C14E12AC097F097530CE0F2
:1014500003EEC9F0D8909735E926000EEA22EECFC8
:1014600084F0EFCF85F003D0856B846B5992B7D0B1
:101470003E0E295C14E12AC098F098530CE003EE6C
:10148000C9F0D8909835E926000EEA22EECF86F012
:10149000EFCF87F003D0876B866B5994A0D03F0EB7
:1014A000295C14E12AC099F099530CE003EEC9F0CD
:1014B000D8909935E926000EEA22EECF88F0EFCFDA
:1014C00089F003D0896B886B599689D0400E295CCE
:1014D00014E12AC09AF09A530CE003EEC9F0D890B8
:1014E0009A35E926000EEA22EECF8AF0EFCF8BF094
:1014F00003D08B6B8A6B599872D0410E295C14E132
:101500002AC09BF09B530CE003EEC9F0D8909B35AA
:10151000E926000EEA22EECF8CF0EFCF8DF003D05B
:101520008D6B8C6B599A5BD0420E295C14E12AC0FA
:101530009CF09C530CE003EEC9F0D8909C35E92652
:10154000000EEA22EECF8EF0EFCF8FF003D08F6B3C
:101550008E6B599C44D0430E295C14E12AC09DF047
:101560009D530CE003EEC9F0D8909D35E926000E9E
:10157000EA22EECF90F0EFCF91F003D0916B906B19
:10158000599E2DD0440E295C14E12AC09EF09E5332
:101590000CE003EEC9F0D8909E35E926000EEA2251
:1015A000EECF92F0EFCF93F003D0936B926B5A9003
:1015B00016D0450E295C13E12AC09FF09F530CE022
:1015C00003EEC9F0D8909F35E926000EEA22EECF4F
:1015D00094F0EFCF95F003D0956B946B5A922968F5
:1015E00012002D5207E1C85304E022EC0EF02DC08A
:1015F000C8F00AD07A0E2D5C07E17A0EC85D04E0CF
:1016000099EC0EF02DC0C8F02D6812001E0E2B5C58
:10161000D8A4A6D02C5221E15A6A596A836B826BF6
:10162000966B856B846B976B876B866B986B896BFE
:10163000886B996B8B6B8A6B9A6B8D6B8C6B9B6BCE
:101640008F6B8E6B9C6B916B906B9D6B936B926BA6
:101650009E6B956B946B9F6B82D02CC096F003EEC3
:10166000C9F0D8902C34E926000EEA22EECF82F0A1
:10167000EFCF83F02CC097F003EEC9F0D8902C3454
:10168000E926000EEA22EECF84F0EFCF85F02CC0E1
:1016900098F003EEC9F0D8902C34E926000EEA2227
:1016A000EECF86F0EFCF87F02CC099F003EEC9F0B3
:1016B000D8902C34E926000EEA22EECF88F0EFCF46
:1016C00089F02CC09AF003EEC9F0D8902C34E926AA
:1016D000000EEA22EECF8AF0EFCF8BF02CC09BF009
:1016E00003EEC9F0D8902C34E926000EEA22EECFA2
:1016F0008CF0EFCF8DF02CC09CF003EEC9F0D890A9
:101700002C34E926000EEA22EECF8EF0EFCF8FF0D8
:101710002CC09DF003EEC9F0D8902C34E926000EC1
:10172000EA22EECF90F0EFCF91F02CC09EF003EEC6
:10173000C9F0D8902C34E926000EEA22EECF92F0C0
:10174000EFCF93F02CC09FF003EEC9F0D8902C346B
:10175000E926000EEA22EECF94F0EFCF95F017D0F5
:10176000420E2B5C07E12C5203E1589012D801D0B5
:1017700058800DD0430E2B5C06E12C5202E18C9276
:1017800001D08C8204D07B0E2B5CD8B43ED82B6861
:1017900012008C92576A566A5A6A596A89928996D7
:1017A000899A8D928A988A948A908C9C8C988B982E
:1017B0008994899089988D908D948A968A928C9E2E
:1017C0008C9A8B9A8C908B96836B826B966B856BC5
:1017D000846B976B876B866B986B896B886B996B47
:1017E0008B6B8A6B9A6B8D6B8C6B9B6B8F6B8E6B21
:1017F0009C6B916B906B9D6B936B926B9E6B956BDF
:10180000946B9F6BC86B22EF0EF0576A566A5A6A48
:10181000596A89928996899A8D928A988A948A902F
:101820008C9C8C988B988994899089988D908D94B4
:101830008A968A928C9E8C9A8B9A8C908B961200A8
:101840000301CA69C969AA0ECC6F480ECB6FA40EFA
:10185000CE6FCC0ECD6FA20ED06F1E0ECF6F9F0E2F
:10186000D26F7C0ED16F9C0ED46FE50ED36F9A0EA3
:10187000D66F590ED56F970ED86FD70ED76F950EBE
:10188000DA6F600ED96F920EDC6FF30EDB6F900E85
:10189000DE6FDD6F8E0EE06F370EDF6F8B0EE26F47
:1018A000E80EE16F890EE46FA20EE36F870EE66F1C
:1018B000660EE56F850EE86F330EE76F830EEA6FF5
:1018C000090EE96F800EEC6FE90EEB6F7E0EEE6F86
:1018D000D10EED6F7C0EF06FC10EEF6F7A0EF26FCE
:1018E000BB0EF16F780EF46FBC0EF36F760EF66FD1
:1018F000C60EF56F740EF86FD90EF76F720EFA6F91
:10190000F30EF96F710EFC6F150EFB6F6F0EFE6F0D
:101910003F0EFD6F6D0E0401006F700E0301FF6F2F
:101920006B0E0401026FA90E016F690E046FEA0EBF
:10193000036F680E066F310E056F660E086F800E1E
:10194000076F640E0A6FD60E096F630E0C6F330EAD
:101950000B6F610E0E6F960E0D6F600E106F010E05
:101960000F6F5E0E126F720E116F5C0E146FE90E28
:10197000136F5B0E166F670E156F590E186FEB0E17
:10198000176F580E1A6F750E196F570E1C6F050ED4
:101990001B6F550E1E6F9B0E1D6F540E206F370E62
:1019A0001F6F520E226FD90E216F510E246F810EC0
:1019B000236F500E266F2E0E256F4E0E286FE10EF0
:1019C000276F4D0E2A6F990E296F4C0E2C6F560EF5
:1019D0002B6F4B0E2E6F190E2D6F490E306FE00ED0
:1019E0002F6F480E326FAD0E316F470E346F7F0E82
:1019F000336F460E366F560E356F450E386F320E0A
:101A0000376F440E3A6F120E396F420E3C6FF70E6D
:101A10003B6F410E3E6FE00E3D6F400E406FCF0EAC
:101A20003F6F3F0E426FC10E416F3E0E446FB80EC6
:101A3000436F3D0E466FB30E456F3C0E486FB30EBD
:101A4000476F3B0E4A6FB60E496F3A0E4C6FBE0E93
:101A50004B6F390E4E6FCA0E4D6F380E506FDA0E47
:101A60004F6F370E526FED0E516F370E546F050EDC
:101A7000536F360E566F200E556F350E586F3F0E52
:101A8000576F340E5A6F620E596F330E5C6F880EAB
:101A90005B6F320E5E6FB20E5D6F310E606FDF0EE8
:101AA0005F6F310E626F100E616F300E646F440E07
:101AB000636F2F0E666F7B0E656F2E0E686FB60E0E
:101AC000676F2D0E6A6FF30E696F2D0E6C6F340EFB
:101AD0006B6F2C0E6E6F780E6D6F2B0E706FBF0ECE
:101AE0006F6F2B0E726F0A0E716F2A0E746F570E86
:101AF000736F290E766FA70E756F280E786FF90E2B
:101B0000776F280E7A6F4F0E796F270E7C6FA80EB5
:101B10007B6F270E7E6F030E7D6F260E806F610E2A
:101B20007F6F250E826FC10E816F250E846F240E8C
:101B3000836F866F8A0E856F230E886FF20E876F14
:101B4000230E8A6F5C0E896F220E8C6FC90E8B6F0D
:101B5000220E8E6F390E8D6F210E906FAA0E8F6F31
:101B6000210E926F1E0E916F200E946F950E936F43
:101B7000200E966F0D0E956F1F0E986F880E976F43
:101B80001F0E9A6F050E996F1E0E9C6F840E9B6F31
:101B90001E0E9E6F050E9D6F1D0EA06F880E9F6F0F
:101BA0001D0EA26F0D0EA16F1C0EA46F950EA36FDC
:101BB0001C0EA66F1E0EA56F1B0EA86FA90EA76F99
:101BC0001B0EAA6F360EA96F1A0EAC6FC50EAB6F47
:101BD0001A0EAE6F560EAD6F190EB06FE80EAF6FE6
:101BE000190EB26F7C0EB16F190EB46F120EB36F77
:101BF000180EB66FAA0EB56F180EB86F440EB76FF9
:101C0000170EBA6FDF0EB96F170EBC6F7B0EBB6F6E
:101C1000170EBE6F1A0EBD6F160EC06FBA0EBF6FD5
:101C2000160EC26F5B0EC16F150EC46FFE0EC36F32
:101C3000150EC66FA30EC56F150EC86F490EC76F80
:101C400000011200010E806F800E805DD8B070D050
:101C50000B6A800E0A6E180E096E880E086E1F0E33
:101C60000F6E850E0E6E370E0D6E820E0C6E80514D
:101C700056EC01F01AC013F019C012F018C011F0A0
:101C800017C010F01E6A1D6A1C6A7F0E1B6E13C0FF
:101C90001AF012C019F011C018F010C017F025EC9E
:101CA00000F01AC013F019C012F018C011F017C0DC
:101CB00010F00FC01EF00EC01DF00DC01CF00CC0C7
:101CC0001BF013C01AF012C019F011C018F010C0A8
:101CD00017F0B5EC00F01AC00FF019C00EF018C0E4
:101CE0000DF017C00CF00BC01EF00AC01DF009C0AB
:101CF0001CF008C01BF00FC01AF00EC019F00DC088
:101D000018F00CC017F027EC00F003EC01F0006EA7
:101D100018C001F002EEC9F0D8908035E926000E17
:101D2000EA2200C0EEFF01C0EFFF802BD8A08CD7C5
:101D30001200010E806F800E805DD8B06FD00B6AEC
:101D40000A6A520E096E850E086E520E0F6EB80E9C
:101D50000E6E130E0D6E840E0C6E805156EC01F05B
:101D60001AC013F019C012F018C011F017C010F00B
:101D70001E6A1D6A1C6A7F0E1B6E13C01AF012C009
:101D800019F011C018F010C017F025EC00F01AC0BF
:101D900013F019C012F018C011F017C010F00FC0E6
:101DA0001EF00EC01DF00DC01CF00CC01BF013C0C7
:101DB0001AF012C019F011C018F010C017F0B5ECED
:101DC00000F01AC00FF019C00EF018C00DF017C0C7
:101DD0000CF00BC01EF00AC01DF009C01CF008C0BA
:101DE0001BF00FC01AF00EC019F00DC018F00CC097
:101DF00017F027EC00F003EC01F0006E18C001F0C2
:101E000002EEC9F0D8908035E926000EEA2200C023
:101E1000EEFF01C0EFFF802BD8A08DD71200FFD7B7
:020000040030CA
:0300010006160ED2
:020005008580F4
:060008000FC00FE00F40E5
:00000001FF
